:100000000AC018951895189518951895189518956B
:100010001895189518950FED0DBF00E008B90FEF72
:1000200002BB0CEF08BB09EB01BB08E107BB0000FA
:100030000000829904C000E50093600021C081990E
:1000400004C004E6009360001BC0B79904C002E836
:100050000093600015C0B69904C006E900936000E3
:100060000FC0B59904C004EB0093600009C0B299B9
:1000700004C006EE0093600003C000E0009360003F
:100080008CE697E0ECE6F7E005E0202E04E6002E93
:1000900095980A94F1F7959A04E6002E0A94F1F7E0
:1000A00006E9002E02E0102E94980A94F1F71A94B3
:1000B000E1F7949A009060000A94F1F700E5002EB1
:1000C00093980A94F1F7939A459901C041C00000B2
:1000D000000000000000000000000000C49A04E1DD
:1000E000081700E0090780F4869905C08350904006
:1000F000ED5FFF4F09C02A9439F481509040EF5FC3
:10010000FF4F05E0202E07C00000000000000000A7
:10011000000000000000682E792E4E2E5F2E909871
:10012000062D0150602E072D0040702E00E00615B0
:1001300000E00705A9F7909A042D0150402E052DE7
:100140000040502E00E0041500E00505A9F79ECF01
:10015000000000000000000000000000000000009F
:100160000000000000000000C49804E10E1700E049
:100170000F0758F4869905C08D5F9F4FE350F040FC
:1001800004C08F5F9F4FE150F040682E792E4E2EB5
:100190005F2E9098062D0150602E072D0040702E86
:1001A00000E0061500E00705A9F7909A042D01501C
:1001B000402E052D0040502E00E0041500E00505FE
:0401C000A9F764CF68
:00000001FF
